:020000040800F2
:100000001807002051030008590300085B0300088B
:100010005D0300085F0300086103000800000000A2
:100020000000000000000000000000006303000862
:10003000650300080000000067030008951D000824
:100040006B0300086B0300086B0300086B030008D8
:100050006B0300086B0300086B0300086B030008C8
:100060006B0300086B0300086B0300086B030008B8
:100070006B0300086B0300086B0300086B030008A8
:100080006B0300086B0300086B0300086B03000898
:100090006B0300086B0300086B0300086B03000888
:1000A0006B0300086B0300086B0300086B03000878
:1000B0006B0300086B0300086B0300086B03000868
:1000C0006B0300086B0300086B0300086B03000858
:1000D0006B0300086B0300086B0300086B03000848
:1000E0006B0300086B0300086B0300086B03000838
:1000F0006B0300086B0300086B0300086B03000828
:100100006B0300086B0300086B0300086B03000817
:100110006B0300086B0300086B0300086B03000807
:100120006B0300086B0300086B0300086B030008F7
:100130006B0300086B0300086B0300086B030008E7
:100140006B0300086B0300086B0300086B030008D7
:100150006B0300086B0300086B0300086B030008C7
:100160006B0300086B0300086B0300086B030008B7
:100170006B0300086B0300086B0300086B030008A7
:100180006B0300086B0300086B0300086B03000897
:100190006B030008000000006B0300086B030008FD
:1001A0006B0300086B0300086B0300086B03000877
:1001B0006B0300086B0300086B0300086B03000867
:1001C0006B0300086B0300086B0300086B03000857
:1001D0006B0300086B03000800F002F800F0A8F8B9
:1001E00014A696E8000CB244B344DA4501D100F0FD
:1001F0009FF8BAE80F000FA696E83000A5EB0405BB
:1002000004EB0607AAEB0704A7F101074FEA15154F
:100210004FEA3414A4F10104AC4201D300F088F891
:1002200013F0010F18BFFB1A43F0010300F001F8AF
:10023000DBE718474433000064330000103A24BF62
:1002400078C878C1FAD8520724BF30C830C144BF3B
:1002500004680C6070470000704700000023002411
:1002600000250026103A28BF78C1FBD8520728BFC6
:1002700030C148BF0B6070476E2900F0B181702912
:1002800000F0E782662902F0C487652902F0C18781
:10029000672902F0BE87612902F0BD8703681B0A47
:1002A00028BF41F08001692900F05E81642900F0D7
:1002B0005B81752900F058816F2900F075827829DB
:1002C00000F0B382E92900F00F82E42900F00C82EB
:1002D000F52900F00982EF2900F07282F82900F078
:1002E000B2820368DB0928BF41F08001632900F076
:1002F000CB87732900F0D087E32900F0DB87F3294F
:1003000000F0E087002070471FB502F075FF01F094
:1003100033F804000020002102F058FF401C606008
:100320000020002102F03CFFE0601FBD10B510BDB1
:1003300000F0F4FF1146FFF7E7FF02F099F901F032
:10034000D1F803B4FFF7F2FF03BC01F04FFE000049
:100350000948804709480047FEE7FEE7FEE7FEE759
:10036000FEE7FEE7FEE7FEE7FEE7FEE70448054995
:10037000054A064B70470000891F0008D901000894
:10038000180100201807002018030020180300207F
:10039000704753EA020C00F069802DE9F04B4FF0F2
:1003A0000006002B1FBFB3FA83F503FA05F424FA05
:1003B00005F65E4012BF1643B2FA82F502FA05F462
:1003C000C5F120051EBF22FA05FC44EA0C042035C5
:1003D00056EA044C4FEA144418BF641C4FF000085E
:1003E0004FF00009904271EB030C39D3002919BF7B
:1003F000B1FA81F701FA07F6B0FA80F700FA07F6CA
:10040000C7F120071EBF20FA07FC46EA0C0620377A
:10041000B6FBF4FCA7EB0507103F07F01F0BCBF171
:1004200020062CFA06F60CFA0BFB44BFB346002656
:10043000202FA4BF5E464FF0000B5BEA060C08BFFE
:100440004FF0010B19EB0B0948EB0608ABFB027CE4
:1004500006FB02CC0BFB03CCC01B71EB0C01C1E70C
:100460000B46024641464846BDE8F08B13B50843AB
:1004700018BF4FF0FF300146AFF30080BDE81C40CD
:10048000704700000FB4044910B503AA029800F0A9
:10049000BBF810BC5DF814FBB0000020704770473B
:1004A0007047704770B5044685690068C10601D57C
:1004B000302600E02026C00707D070BDD4E9012116
:1004C00030469047206A401C20626D1EF6D570BDF4
:1004D00070B5044685690078C00707D170BDD4E9BE
:1004E000012120209047206A401C20626D1EF6D515
:1004F00070BD09684A0501D540B27047C905FCD5F1
:1005000000B2704709684A0501D5C0B27047C905F5
:10051000FCD580B2704770B50C460546012A05D05F
:100520002878800600D5EA69002302E0012305E06F
:100530005B1C934202D2E05C0028F9D1A869E6185E
:10054000C01AA861286A184428622846FFF7AAFF43
:1005500004E0D5E9012114F8010B9047B442F8D327
:100560002846FFF7B5FF70BD2DE9F041064600248F
:1005700010687529314616A510D0FFF7BAFF00287C
:1005800002DA404213A507E031688A0701D512A5B7
:1005900002E0490704D511A5012401E0FFF7B2FFED
:1005A00000210A2206F1240709E0B0FBF2FCB0FBAF
:1005B000F2F302FB1C00303078541846491C002826
:1005C000F3D123462A463046BDE8F04100F055BA43
:1005D000000000002D0000002B00000020000000A3
:1005E00011680268006A530501D508700AE0D30556
:1005F00001D5088006E0130603D5C217C1E9000241
:1006000000E0086001207047074B70B50D467B4441
:1006100000F01DFE0446284600F058FE10B14FF0D1
:10062000FF3070BD204670BD2F1B00002DE9FF5F1D
:1006300015468A460446DFF8AC80F8440027D8E91E
:1006400000103E46CDE9001010E03AF816106A4658
:1006500002A800F03FFE411C07D02178890603D58F
:10066000E269391891420DD80744761C207880063B
:1006700002D5E069B84205DDAE42E6DB3AF8160085
:100680000028E2D1A069C01BA0612046FFF70AFF45
:10069000D8E90010CDE90010002017E03AF8181052
:1006A0006A4602A800F016FEB0F1FF3F81460BD06B
:1006B00000250DF1080B05E0D4E901211BF8050028
:1006C00090476D1C4D45F7D308F10100B0428046BC
:1006D000E4DB206A384420622046FFF7F9FEBDE8DB
:1006E000FF9F0000DE2B00002DE9F0418046D21D67
:1006F00022F007020025D2E90002F52915A614D040
:10070000011E72F1000106DA0023D0EB030063EB57
:10071000020211A608E0D8F800108B0701D50FA639
:1007200002E0490701D50EA601251146002408F173
:10073000240704E000F05CF930323A55641C50EABA
:100740000102F7D12B46324621464046BDE8F04132
:1007500000F093B9000000002D0000002B00000005
:100760002000000030B4002100F1240408E002F071
:100770000705D208303542EA4372DB086554491C4C
:1007800052EA0305F3D10468002310A2250708D517
:1007900004F020040C4304D0C46901230CA2641E9D
:1007A000C46130BC00F069B910B504462146106838
:1007B000FFF7A8FE02462046BDE810400023D1E71F
:1007C000D21D22F00701D1E90023CBE70000000091
:1007D00030000000F0B40D460188090502D5214C17
:1007E0007C4402E01F4C7C440E34002100F12406BE
:1007F00008E002F00F071209E75D42EA03721B09E5
:100800007754491C52EA0307F3D1027800231207F8
:1008100004D5702D06D009B1022311342246F0BC54
:1008200000F02BB901231034F8E770B504460D46EB
:1008300021461068FFF766FE024629462046BDE8BD
:1008400070400023C6E7D21D22F00703D3E900233E
:10085000C0E70368126843F0200303600823C36104
:100860000023B7E7402A00002DE9F05F89460446DF
:100870004FF0000ADFF874B1FB44C0F820A0204616
:10088000E1688847002874D0252806D0D4E90121E2
:100890009047206A401C2062F1E700265F46204610
:1008A000E16888472028054607DB312D05D27819F5
:1008B00010F8200C08B10643F1E7B00701D526F087
:1008C0000406C4F81CA00027C4F818A02A2D09D0DB
:1008D000284602F05DFC38B304EB8708303DC8F8C9
:1008E000185019E059F8041B204604EB8702916167
:1008F000E1688847012F054618D1E069002820DA11
:1009000026F020061DE0D8F8180000EB800005EB6B
:1009100040003038C8F818002046E168884705468E
:1009200002F036FC0028EED1012F0AD02E2D08D17E
:100930002046E16888477F1C0546022F46F02006C6
:10094000C4DBA069002803DA404246F00106A0613A
:10095000F00701D026F010066C2D0BD0682D09D0C1
:100960004C2D39D06A2D35D0742D35D07A2D33D019
:1009700016E038E0E1682F4620468847B842054631
:1009800009D16C2F26D04FF48060E16806432046E1
:100990008847054604E06C2F1AD04FF48070064358
:1009A0000DB3A5F14100192802D8203546F40066A0
:1009B0004A462946204626604E46FFF75DFC80B138
:1009C00001280BD0F61D26F0070000F1080956E7B4
:1009D0004020E4E78020D8E70020D6E706F10409AC
:1009E0004DE7284652E7206ABDE8F09FD029000075
:1009F00030B5B0F10A0271F100034FEA900E4EEAF1
:100A0000817EB0EB0E0061EB91014FEA101E4EEAC1
:100A1000017E10EB0E0041EB11114FEA102E4EEA51
:100A2000016E10EB0E0041EB11214FEA104E4EEA21
:100A3000014E10EB0E0041EB1141401841F1000155
:100A40004FEAD00040EA41704FEAD1014FEA8104F9
:100A500044EA907410EB800544EB01046D1944EBFB
:100A60000404521BA3414FF0000348BF0A3200D5D3
:100A700030BD401C41F1000130BD2DE9F0470D466D
:100A800099469246044600F124080168880604D578
:100A9000E06921F01001216000E00120A84201DDA1
:100AA000471B00E00027A1697A1902EB0900081A28
:100AB000A0612078C00602D42046FFF7F3FC002690
:100AC00008E0D4E901211AF806009047206A401C8A
:100AD000761C20624E45F4DB2078C0060AD52046FD
:100AE000FFF7E0FC06E0D4E9012130209047206ABE
:100AF000401C2062381EA7F10107F4DC07E0D4E9AE
:100B0000012118F805009047206A401C2062281E29
:100B1000A5F10105F3DC2046FFF7DAFC207800069A
:100B200002D50220BDE8F0870120FBE72DE9FF4F49
:100B30000C461E464FF0FF378BB0D2E90001DDF8BE
:100B400060800A908A46C1F30A5505B93D460021E6
:100B500008464FF00000BAF1000F00F4400005DA3B
:100B600000EB80004FF4400101EA50004FEA905939
:100B7000B9F1010F00DDB9460A9850EA4A000ED0DB
:100B800044F61050A5F2FF3545432F14B8F1000F7D
:100B90001ED07542291E1EDDC9F100021CE0B8F10D
:100BA000010F4FF0000001D0302103E0F24305E0D7
:100BB0002154401CB042FBDB30460022002121546E
:100BC0000B99C1F80880C1E900200FB0BDE8F08F93
:100BD000BD1B6D1CDEE74A4600DA694206A800F03C
:100BE0000FFC06AB93E8070003AB83E80700504611
:100BF0000A9901F0EDFE8DE80700A0F500501F38BE
:100C000000900398002D0ADD42F21F014A46084475
:100C1000002303A90390684602F056F909E0A0F505
:100C200000504A461F38002303A90390684602F08B
:100C300060F98DE807000004000C03D04FF0FF308E
:100C4000410800E01046B8F1000F03D000220092E6
:100C500015461EE0751E05D4FFF7CAFE30326255F8
:100C60006D1EF9D5B3460122084302D000227F1C35
:100C700004E02078302801D100227F1E002A099745
:100C800084D01DE0112D07DAFFF7B2FE3032625535
:100C90006D1C50EA0102F5D1084302D00098C8B19A
:100CA0000EE00021681E05E0235C625C6354225460
:100CB000401E491C8142F7DBAB46A81B401E099031
:100CC000002004F80B000B98099AC0F80880C0E9CE
:100CD000002B7AE711264FF0000857E72DE9F04F77
:100CE00088460446D21D22F0070191B0D1E90001E7
:100CF000CDE90A0102F034FA02460B98C00F01D088
:100D00002D2007E02068810701D52B2002E020215B
:100D100001EAC000032A099001D0072A05DB034637
:100D20004146204600F02CFB0BE12078800601D5DF
:100D3000E06900E00620B8F1650F814606D0B8F101
:100D4000660F18D0B8F1670F70D131E00020B9F10B
:100D5000110F009001DB112301E009F101030AAA40
:100D600001A90CA8FFF7E2FEDDE90C70002609F1ED
:100D70000105834647E001204B4600904FF00047B5
:100D80000AAA01A90CA8FFF7D1FEDDE90DB00C9964
:100D90005D46002610B909F101000D18B9EB0500F8
:100DA00003D4C0F1FF3609F10105A5EB09002BE0E2
:100DB000B9F1010F01DA4FF001090020B9F1110F6B
:100DC0000090484601DD112300E003460AAA01A96C
:100DD0000CA8FFF7ABFEDDE90C704D4600268346FC
:100DE000207800070AD4AB4500DA5D4601A8012D42
:100DF00004DD411911F8011C302907D04F4502DAF2
:100E000017F1040F04DA012082460FE06D1EEEE7B1
:100E1000002F02DCED1B3E4403E0781CA84200DDFD
:100E20007D1CB81B00F1010A4FF000472078000735
:100E300003D4AA4501DB4FF0FF3A0021B7F1004F80
:100E40000DF143088DF8431024D002202B23002FEE
:100E500001DA7F422D230A21021EA0F1010000DCED
:100E60005FB197FBF1FC97FBF1F201FB1C7C17468D
:100E70000CF1300C08F801CDEEE7A8F10100037089
:100E80002188090501D5452100E06521A0F101086F
:100E900000F8011C09980FA9A1EB0807FF1D00B17C
:100EA0000120411901EBEA70A1693844081A401E7B
:100EB000A0612078C00602D42046FFF7F3FA099813
:100EC00028B1D4E901219047206A401C2062207893
:100ED000C00622D52046FFF7E5FA1EE0002E04DB0F
:100EE000B34502DD01A8805D00E03020D4E9012196
:100EF0009047206A401C2062761CAAF101005FEA3C
:100F0000000A0AD100F038FAC0680168405CD4E9F0
:100F100001219047206A401C2062281EA5F101058E
:100F2000DCDC07E0D4E9012118F8010B9047206AC6
:100F3000401C2062381EA7F10107F3DC2046FFF7B2
:100F4000C7FA032011B041E62DE9F04F04460D46E3
:100F5000D21D22F0070089B0D0E9009748463946F3
:100F600002F0FEF80246F80F01D02D2307E02068BA
:100F7000810701D52B2302E0202101EAC0038DF86F
:100F800020300BB1012000E00020032A824601D06E
:100F9000072A04DB2946204600F0F2F93FE12078D9
:100FA000800601D40D2500E0E569C7F30A560D2D32
:100FB00049DA00214FEA175B08464FF00000002F86
:100FC00000F4400007DA00EB80004FF4400100EB32
:100FD000D07001EA60008115012901DD4FF0FF3179
:100FE00000224FEA850CBCF1180F06D31346ACF172
:100FF00018004FF08052C24003E04FF4801323FAF0
:101000000CF30CF10C0CBCF1200F04D3ACF1200C50
:1010100009FA0CF001E007FA0CF000294FF0004843
:1010200001DD18B90FE00ED140450CD319EB0209D0
:101030005F4121B9404502D19F4329EA0209BBEB38
:10104000175F00D0761C2088000502D57B487844C5
:1010500002E07A487844193808AA302302F80A30A6
:10106000037C0AF10101002E0AF1020A53546A4678
:1010700002DC4FF0300101E04FF031014FF0010888
:101080008DF8001002D0A6F2FF3603E059EA4701BE
:1010900000D06B4E002D02DC2178090704D54FF0FB
:1010A00002082E218DF80110C44600210BE0C7F381
:1010B00003433F01C35C491C6D1E02F8083005293B
:1010C00008F1010801DA002DF1DC00210CE000EB51
:1010D0001973491C1B786D1E082902F808304FEA65
:1010E000091908F1010801DA002DF0DC21688B06EE
:1010F00002D516E0A8F10108E04505DD02EB080382
:1011000013F8013C302BF5D0B8F1000F09DD02EBEC
:10111000080313F8013C2E2B03D1090701D4A8F1D1
:101120000108002D05DD3E2102F808106D1E08F1B2
:101130000108407C002E02F8080008F1010804DADA
:101140002D20764202F8080002E02B2002F8080069
:101150000A214FF47A70864208F101080BDB96FBF6
:10116000F0F3303302F8083096FBF0F308F1010891
:1011700000FB136601E0642E0CDB642096FBF0F3A9
:10118000303302F8083096FBF0F308F1010800FB59
:10119000136601E00A2E06DB96FBF1F0303002F810
:1011A000080008F1010896FBF1F001FB10603030F7
:1011B00002F80800A16908F1010808EB050202EB3A
:1011C0000A00081AA0612078C00602D42046FFF762
:1011D00069F9216A08AE01EB0A00206204E0D4E953
:1011E000012116F8010B9047BAF1010AF7D22078D5
:1011F000C00602D52046FFF755F96E4609E016F8FD
:10120000010B3E280FD0D4E901219047206A401CF1
:101210002062B8F10108F2D22046FFF759F909B06F
:101220000320BDE8F08F206A2844206203E0D4E95F
:101230000121302090476D1EEBD3F8E71E220000FD
:1012400002FCFFFF01694A1C02610878704700B583
:101250008FB0CDE901310021059105497944CDE9EF
:10126000031011466846FFF7FFFA0FB000BD0000FB
:10127000E5FFFFFF10B5436913B1AFF3008001E054
:10128000FFF749F9012010BD127800F124010A701E
:1012900000224A700122EDE711684FF0FF32E9E7C2
:1012A00010B5436913B1AFF3008001E0FFF7BEF959
:1012B000012010BD128800F1240182840022C28422
:1012C0000122EDE711684FF0FF32E9E7007B00F003
:1012D000800070472DE9F04116460C46054600F0A7
:1012E00043F8036893F80101012807D0FF2C12D8B6
:1012F000185D80B101202C70BDE8F081D3F80701A2
:101300003246214603F20713C7182846BC46BDE8FB
:10131000F041002360474FF0FF30EDE7754600F0E5
:10132000EBF8AE4605006946534620F007008546B7
:1013300018B020B5FFF71AF8BDE820404FF00006BE
:101340004FF000074FF000084FF0000BAC46ACE840
:10135000C009ACE8C009ACE8C009ACE8C00921F09C
:1013600007018D467047000010B500F005F8001D1C
:1013700010BD00BF591E00000048704770000020DB
:101380002DE9F0411F46044603260168072A01F4AF
:10139000006004DB08B116A505E016A503E008B15E
:1013A00015A500E015A521F010002060A069C01E61
:1013B000A0610FB1401EA0612046FFF773F84FB146
:1013C000D4E9012138469047206A401C2062C01CA5
:1013D000206206E0206AFAE7D4E9012115F8010B42
:1013E0009047761EF8D22046FFF772F8BDE8F081EC
:1013F0004E414E006E616E00494E4600696E6600B9
:101400002DE9F047814616468AB0354878440DC824
:101410008DE80D0032487844801C03AC0DC884E888
:101420000D0041F69B300844372190FBF1F290FB10
:10143000F1F5A5F1800501FB12041B3C02D56442C5
:10144000012000E00020DFF898A080460027FA4441
:10145000AAF1BE0A0EE0E0070AD03246684607EB62
:10146000470101230AEB810101F043FD8DE80700EC
:1014700064107F1C002CEED1194F7F44AE3F19E061
:10148000E80715D007EB04100DF1180A90E80E00DC
:101490008AE80E00C068F04201D1981908903246DF
:1014A000012306A903A801F024FD03AB83E807008C
:1014B0006D10641C002DE3D14FF0010332466946E4
:1014C000B8F1000F03A802D001F0FEFC01E001F02A
:1014D00010FDC9E90001C9F808200AB0BDE8F0878D
:1014E000F01E000010B50446AFF300802046BDE8B2
:1014F0001040FEF726BF0000004870475000002053
:1015000030B44FF0013C50F8042B51F8043BCCFAB6
:1015100052F4D51A20D1FCB950F8042B51F8043BF1
:10152000CCFA52F4D51A17D1B4B950F8042B51F8AB
:10153000043BCCFA52F4D51A0ED16CB950F8042BF6
:1015400051F8043BCCFA52F4D51A05D1002CDAD06C
:1015500030BC4FF00000704729BAB1FA81F111F0A8
:101560001801D1F120008440F2D1CA40CB4012F0E2
:10157000FF0213F0FF0330BCD01A704780B582B071
:10158000019000F02BF80090FFE700F027F8009999
:10159000401A0199884202D2FFE700BFF5E702B086
:1015A00080BD000072B6FFE700BFFDE780B500F028
:1015B000F9FB40F20000C2F20000006844F6D3518B
:1015C000C1F26201A0FB0110800900F0B9FB18B163
:1015D000FFE7FFF7E7FFFFE780BD000040F20C10D8
:1015E000C2F200000068704780B541F20000C4F20A
:1015F0000200016841F4807101604FF4806101F0E4
:1016000097F9002000F01EFB41F20800C4F202002E
:10161000012101600C21042201F0B2F900F04CFC20
:1016200080BD000080B540F20510C2F200000078D5
:10163000C00708B9FFE713E000F042FE40F21010C7
:10164000C2F20000007802280AD1FFE740F204004D
:10165000C2F20000C06801F0E9F800F091FEFFE777
:1016600080BD000080B58AB005A800F08BF940F27B
:101670001010C2F200000078032801D0FFE7BAE0A2
:10168000079840F20401C2F20001496A884204D27C
:10169000FFE7012000F0C6FFADE0099840F2040129
:1016A000C2F20001896A884204D9FFE7022000F0F3
:1016B000B9FFA0E0089840F20401C2F20001096BF2
:1016C000884204D9FFE7032000F0ACFF93E040F22A
:1016D0000400C2F200000190006A40F24801C2F228
:1016E00000010968A0FB0101079A0023FEF751FEE3
:1016F00001990390086A099A801A04900498896BEA
:10170000484348F21F51C5F2EB1150FB01F148115B
:1017100000EBD17240F20810C2F2000001681144DF
:101720000160006840F6B931884208DBFFE740F20B
:101730000811C2F2000140F6B830086016E040F22D
:101740000810C2F2000000684FF24741CFF6FF7167
:1017500088420ADCFFE740F20811C2F200014FF2B2
:101760004840CFF6FF700860FFE7FFE70398049A50
:1017700040F20401C2F200014B6B5A4348F21F537E
:10178000C5F2EB1352FB03F35A1102EBD372104470
:1017900040F20812C2F20002126810440290089847
:1017A000C96A88420DD9FFE7089840F20401C2F2E5
:1017B0000001CA6A801AC96B029A00FB11200290CC
:1017C000FFE70298B0F1FF3F03DCFFE70020029043
:1017D0000DE00298009000F0B1FE014600988842AA
:1017E00004DDFFE700F0AAFE0290FFE7FFE70298A2
:1017F00000F0C6FDFFE70AB080BD000083B08DF8A1
:1018000007009DF8070001460091042823D800999D
:10181000DFE801F003090F151B0043F21A50C0F670
:10182000000002901DE043F2F840C0F60000029074
:1018300017E043F20950C0F60000029011E043F2B5
:101840004950C0F6000002900BE043F26450C0F62D
:101850000000029005E043F22750C0F6000002901D
:10186000FFE7029803B0704740F24400C2F2000064
:101870000068704740F20410C2F200000078704720
:1018800081B040F20400C2F200000068C0B2022839
:1018900008D8FFE740F20400C2F2000000688DF8AB
:1018A000030003E000208DF80300FFE79DF803002C
:1018B00001B0704740F24800C2F200000068704773
:1018C00040F21010C2F200000078704780B500F0BE
:1018D0004BFC002000F0EEFF00F0E4FF00F08CFB7A
:1018E00000F074FD014640F20510C2F200000170E4
:1018F0000078C00720B1FFE7002000F029FDFFE7D6
:1019000040F21011C2F200010120087040F20411EF
:10191000C2F200010020087080BD000040F20510F6
:10192000C2F20000007800F00100704783B08DF82B
:1019300007009DF807000146009140B1FFE70098BD
:1019400001280AD0FFE7009802280CD011E043F2EA
:101950003B50C0F60000029011E043F25B50C0F62D
:10196000000002900BE043F22F50C0F600000290FE
:1019700005E043F22750C0F600000290FFE702980E
:1019800003B0704780B586B00590022000F088FB58
:1019900005990880032000F083FB05994880042006
:1019A00000F07EFB059988800598008800F09EFB7A
:1019B00004900598408800F099FB03900598808872
:1019C00000F094FB0290049840F68B01C0F20301F2
:1019D000019100F055FF05998860039800F040FFE1
:1019E0000199059AD060029800F04AFF05990861B4
:1019F00006B080BD80B582B0FFF742FF8DF80700CA
:101A0000FFF710FE9DF807000146009140B1FFE787
:101A10000098012818D0FFE70098022820D036E06F
:101A200040F21010C2F200000078022808D0FFE750
:101A300040F21010C2F200000078032803D1FFE743
:101A400000F0E4F8FFE723E040F21010C2F20000DB
:101A50000078022803D0FFE700F05AF8FFE717E00C
:101A600040F21010C2F200000078032803D0FFE714
:101A700000F010F8FFE740F21010C2F2000000780A
:101A8000032803D1FFE7FFF7EDFDFFE700E0FFE7E5
:101A900002B080BD80B540F20410C2F200000078B0
:101AA00008B1FFE733E040F20510C2F20000007811
:101AB000C00720B9FFE7042000F0B4FD27E040F2A2
:101AC0000400C2F200004068002818BF012000F0A6
:101AD000F1FE40F20811C2F200010020086000F09F
:101AE000EFFB4FF4C87000F04BFC46F60001C4F267
:101AF0000101086840F400200860012000F028FC83
:101B000040F21011C2F2000103200870FFE780BD0F
:101B100080B582B040F20410C2F20000007808B133
:101B2000FFE73AE040F20510C2F200000078C0077B
:101B300020B9FFE7042000F075FD2EE000F0C0FBA7
:101B400040F20400C2F20000C06800F06FFE019095
:101B5000019818B9FFE701200190FFE700200090ED
:101B600000F0A8FE009840F20811C2F200010860DF
:101B7000019800F005FC46F60001C4F20101086876
:101B800040F400200860012000F0E2FB40F2101158
:101B9000C2F2000102200870FFE702B080BD000021
:101BA00083B08DF807009DF80700014600910428D6
:101BB00023D80099DFE801F003090F151B0043F259
:101BC000F040C0F6000002901DE043F2EA40C0F68B
:101BD0000000029017E043F25B50C0F60000029054
:101BE00011E043F21F50C0F6000002900BE043F2F8
:101BF0004350C0F60000029005E043F22750C0F6C3
:101C000000000290FFE7029803B0704780B582B0F1
:101C10000020019000F09CFB019800F0B1FB0198BE
:101C200046F60002C4F20102116821F4002111609D
:101C300000F040FE019840F21011C2F2000108705D
:101C400002B080BD83B0029044F24020C0F20F0089
:101C5000019042F20001C4F20201086820F00F0076
:101C6000029A10430860FFE742F20000C4F202004B
:101C7000006800F00F01029A00209142009006D007
:101C8000FFE70198002818BF01200090FFE70098A7
:101C9000C00720B1FFE7019801380190E4E70198FF
:101CA000002818BF012003B07047000080B582B043
:101CB000019000F0CBFA41F25800C4F20200016832
:101CC00041F480210160006844F60001C4F2000183
:101CD0000020086044F60402C4F20002106044F6DA
:101CE0000802C4F20002106040F20000C2F20000DC
:101CF0000068019A00EB5200B0FBF2F044F60C02CF
:101D0000C4F2000210600D20086002B080BD000027
:101D100081B08DF80300FFE744F61C00C4F2000018
:101D200000680006002802D4FFE700BFF4E79DF832
:101D3000030044F62801C4F20001086001B07047B6
:101D400080B582B0009000980138B0F1807F03D355
:101D5000FFE70120019019E0009801384EF21401CC
:101D6000CEF2000108604FF0FF300F2100F01CF9A7
:101D70004EF21801CEF20001002008604EF210026F
:101D8000CEF20002072111600190FFE7019802B036
:101D900080BD000040F20C11C2F200010868013061
:101DA0000860704780B5FFF71FFC41F25800C4F28D
:101DB0000200016841F080510160006847F20001B3
:101DC000C4F200010868012262F34A20086047F269
:101DD0008001C4F20001086820F48070086047F2B6
:101DE0001400C4F200004FF4806100F07BFD18B9CC
:101DF000FFE7FFF7F9FB5DE00420FFF723FF18B9C9
:101E0000FFE7FFF7F1FB55E041F20000C4F20200EA
:101E1000016841F4807101604FF4806100F088FD39
:101E200018B9FFE7FFF7E0FB44E041F20000C4F21D
:101E30000200016821F0807101604FF0007100F034
:101E400051FD18B9FFE7FFF7CFFB33E041F20C017A
:101E5000C4F2020145F23250C0F20010086041F2B3
:101E60000000C4F20200016841F0807101604FF08F
:101E7000007100F05DFD18B9FFE7FFF7B5FB19E051
:101E800041F20800C4F20200032101600C22114655
:101E900000F076FD18B9FFE7FFF7A6FB0AE042F273
:101EA0000001C4F20201086840F4E060086000F03C
:101EB00003F8FFE780BD000088B042F20040C0F2A6
:101EC000F400079041F20800C4F20200006800F03C
:101ED0000C00069006980C2835D1FFE742F200402E
:101EE000C0F2F400059041F20C00C4F20200006858
:101EF00004909DF81010012000EB1110039004983D
:101F0000C0F3062002900498C0F34160019001994B
:101F1000022000EB41000090049800F00300032829
:101F200006D1FFE741F20020C0F27A000590FFE7FA
:101F300005980399B0FBF1F0029948430099B0FB72
:101F4000F1F007900AE00698082806D1FFE741F271
:101F50000020C0F27A000790FFE7FFE7079841F200
:101F60000801C4F202010968C9B20A0943F2183132
:101F7000C0F60001895CC84040F20001C2F20001D5
:101F8000086008B0704700004EF68851CEF200019C
:101F9000086840F4700008604EF60851CEF2000167
:101FA0004FF000600860704782B08DF80700009124
:101FB0009DF9070000280AD4FFE7009800019DF969
:101FC00007104EF20042CEF2000288540BE0009857
:101FD00000019DF8071001F00F014EF61452CEF2E9
:101FE00000028854FFE702B07047000081B0009003
:101FF000FFE700BFFDE7000080B582B041F24C0072
:10200000C4F20200016841F400510160006840F22E
:102010000831C5F20001086840F44030086008212A
:10202000C5F200010191086820F0005008600868BE
:1020300040F0805008600120FFF7A0FA019908687D
:1020400040F000400860FFE70820C5F2000000688B
:10205000C00F10B1FFE700BFF6E70C21C5F2000189
:102060004FF4805008601421C5F2000145F640305D
:1020700008604FF0A041012008600821C5F200016E
:10208000086840F001000860FFE74FF0A0400068DA
:10209000C00710B9FFE700BFF7E702B080BD00003E
:1020A00081B00090009880013021C5F200010860E5
:1020B0004FF0A0410C2008600821C5F2000108681B
:1020C00040F004000860FFE74FF0A04000684007C0
:1020D000002802D4FFE700BFF6E74020C5F2000069
:1020E00000686FF31F3001B07047000081B0ADF899
:1020F0000200BDF8020040F6E44148431121C1F25C
:102100000101A0FB0110000A01B0704784B00290E9
:102110000191009202980199884203D2FFE7019849
:1021200003900AE002980099884203D9FFE70098DB
:10213000039002E002980390FFE7039804B0704711
:1021400080B582B00190009101980A2804D1FFE780
:102150000D20FFF7DDFDFFE79DF80400FFF7D8FD38
:10216000019802B080BD000041F24C00C4F20200B0
:10217000016841F00701016000684FF09041086874
:1021800040F0FC0008600C21C4F60001086820F053
:10219000FC00086040F20041C4F60001086820F02D
:1021A00070600860086840F02060086040F20441F8
:1021B000C4F60001086820F44050086040F208416D
:1021C000C4F60001086840F07060086040F20C41FD
:1021D000C4F60001086820F07060086040F22441F5
:1021E000C4F60001086820F47F000860086840F425
:1021F0005D00086040F60001C4F6000108684FF673
:102200003F72C0F6FF721040086008684023C5F2B4
:1022100000031843086040F60401C4F60001086892
:102220004CF208039843086040F60801C4F6000128
:1022300008688023CAF200031843086040F60C01C6
:10224000C4F60001086810400860704741F24C0075
:10225000C4F20200016841F004010160006840F628
:102260000001C4F60001086820F4700008600868E6
:1022700040F42000086040F60401C4F6000108683C
:1022800020F44060086040F60801C4F600010868C8
:1022900040F47000086040F60C01C4F600010868C4
:1022A00020F47000086040F62401C4F600010868BC
:1022B00020F47F400860086840F4EE4008607047F2
:1022C00080B588B046F68010C4F20100079040F255
:1022D0000400C2F200000390806800F05DF901463E
:1022E0000398069180690021019140F2FF12029249
:1022F000FFF70CFF0199029A034603980593C06902
:10230000FFF704FF014603980491069940F2480242
:10231000C2F2000211600699079A51610599049A68
:1023200041EA024141F44061079A9163406930B14A
:10233000FFE70799486E40F48070486605E007990A
:10234000486E20F480704866FFE708B080BD00004A
:1023500081B08DF803009DF80300C00738B1FFE796
:1023600046F69431C4F201013020086006E046F6DA
:102370009831C4F2010130200860FFE701B07047D6
:1023800080B582B001900198002803D2FFE70020B9
:1023900001900DE00198009000F0D0F801460098FF
:1023A000884204D9FFE700F0C9F80190FFE7FFE792
:1023B000019846F69C11C4F201010860019840F2B0
:1023C0004401C2F20001086002B080BD80B584B053
:1023D00046F68010C4F20100029041F26000C4F29F
:1023E0000200016841F080610160006841F2400133
:1023F000C4F20201086840F080600860086820F0BC
:102400008060086046F69831C4F20101302008600F
:1024100040F20400C2F20000806800F0BDF840F213
:102420004801C2F20001086046F68C31C4F2010195
:102430004FF48030086046F6CC31C4F201010B2025
:10244000086000F055F890B9FFE746F69831C4F2FD
:1024500001013020086046F60001C4F2010108685D
:1024600020F40020086000208DF80F003BE0029966
:1024700008200090086040F24800C2F200000068A6
:102480000299486102990020019088610299C8610F
:1024900000F054F8009A01460198029B5962029B91
:1024A0004FF47A719962029B0421D963029B1A64EA
:1024B000029B5A64029A916402994866FFF700FFF2
:1024C00046F6BC31C4F201014FF40010086046F634
:1024D0000001C4F20101086820F400200860012016
:1024E0008DF80F00FFE79DF80F0004B080BD0000DD
:1024F00082B044F24020C0F20F000190FFE746F6A0
:102500008830C4F2010001680020C903002900904E
:1025100006D4FFE70198002818BF01200090FFE7CC
:102520000098C00720B1FFE7019801380190E6E765
:102530000198002818BF012002B0704780B582B012
:1025400040F20400C2F20000006901214FF47A72E7
:10255000FFF7DCFD0190019800F068F9009040F26F
:102560004800C2F2000000680B2812D3FFE7009871
:1025700040F24801C2F2000109680139884208D3DB
:10258000FFE740F24800C2F2000000680138009006
:10259000FFE7009802B080BD80B586B00590059831
:1025A00030B9FFE740F64050C0F203000590FFE766
:1025B00040F20000C2F20000D0F800E04FEADE6115
:1025C000059A002300935FEA530C4FEA320010EBA8
:1025D0004E1041EB0C01FDF7DCFE02460098019223
:1025E0000A46019903920291029A0399D2F1630279
:1025F000884105D3FFE700200390642002900EE09D
:1026000002990398B1F5803170F1000006D3FFE71D
:10261000002003904FF6FF700290FFE7FFE702985B
:1026200006B080BD80B582B08DF807000020009014
:10263000FFF78EFE0098FFF7A3FE009846F6000213
:10264000C4F20102116821F40021116000F032F996
:102650009DF8070040F20411C2F20001087040F238
:102660001011C2F200010420087002B080BD000009
:102670002DE9F04399B00020189017901690FEF7BE
:1026800095FF4FF4E1300F90FFF710FBFFF71EF9B5
:1026900043F24340C0F60000FDF7F4FE0F9943F209
:1026A000A130C0F60000FDF7EDFE40F20000C2F2DE
:1026B0000000016843F2C340C0F60000FDF7E2FEEF
:1026C000FFF7F8F8024643F2D230C0F6000040F6B9
:1026D0004051C0F20301FDF7D5FEFFF71FF9024696
:1026E00043F2EA40C0F6000043F2DC41C0F60001CC
:1026F000002A18BF014643F2C330C0F60000FDF7C0
:10270000C1FEFFF7BDF8FFF711F9014643F228308B
:10271000C0F60000FDF7B6FE40F2040CC2F2000C59
:10272000DCF80810DCF80C20DCF81430DCF81800B9
:10273000DCF81CE0EC46CCF804E0CCF8000043F2F6
:10274000F730C0F60000FDF79DFE43F25D30C0F6A5
:102750000000FDF797FEFFE7FEF740FF1590159884
:102760001799401A28B1FFE715981790FFF742F91B
:10277000FFE715981699401AB0F5FA7F55D3FFE791
:102780001598169010A8FFF7FDF8FFF779F8FFF7F6
:10279000CDF80990FFF794F8FFF702FA0A90FFF7D7
:1027A00069F8FFF72BF80B90FFF7B8F8024643F2F1
:1027B000EA41C0F6000143F2E640C0F60000002AFC
:1027C00018BF08460D9012980C90139C149DFFF7AB
:1027D0004BF80646FFF76EF809990A9A0B9BDDF84D
:1027E00030E007460D9840F2040CC2F2000CDCF811
:1027F0001880DCF81C90EC46CDF838C0CCF81C9062
:10280000CCF81880CCF81470CCF81060CCF80C50D0
:10281000CCF80840CCF804E0CCF8000043F2684063
:10282000C0F60000FDF72EFEFFE795E780B584B007
:1028300003900398002102914FF47A720192FFF7FE
:1028400065FC019A029B039040F24800C2F200002E
:1028500000680399A0FB0101FDF79BFD04B080BD5A
:1028600081B0009000984FF47A7148434BF69B5129
:10287000CBF2CA51A0FB0110400A01B07047000022
:1028800080B582B001900091019844F24021C0F2DD
:102890000F01A0FB0101009A0023FDF77AFD02B0B1
:1028A00080BD000040F62801C4F600014FF440400E
:1028B0000860704781B08DF803009DF80300C007E1
:1028C00038B1FFE740F61801C4F60001082008609F
:1028D00006E040F62801C4F6000108200860FFE782
:1028E00001B0704784B00390029144F24020C0F2DE
:1028F0000F000190FFE703980168029A002011423F
:10290000009006D0FFE70198002818BF0120009032
:10291000FFE70098C00720B1FFE701980138019058
:10292000E9E70198002818BF012004B070470000B3
:1029300084B00390029144F24020C0F20F00019055
:10294000FFE703980068029A00EA02010020914222
:10295000009006D0FFE70198002818BF01200090E2
:10296000FFE70098C00720B1FFE701980138019008
:10297000E7E70198002818BF012004B07047000065
:1029800085B004900391029244F24020C0F20F00FF
:102990000190FFE70498006803990140029A002023
:1029A0009142009006D0FFE70198002818BF01204F
:1029B0000090FFE70098C00720B1FFE701980138B9
:1029C0000190E7E70198002818BF012005B0704783
:1029D0005FEA400C08BF91F0000F4FEA8C234FEAEA
:1029E000C12243EA51514FEA1C5018BF00F5F04094
:1029F0004FEA300018BF41F000415FEA6C5C00F024
:102A00002980BCF1FF3F08BF40F080407047130CA5
:102A100006BF12044FF0100C4FF0000C130E04BF51
:102A200012020CF1080C130F04BF12010CF1040C7C
:102A3000930F04BF92000CF1020CD30F04BF52009D
:102A40000CF1010C11464FF00002A0F11F00A0EBA9
:102A50000C00704711F0004F08BF704731F0004183
:102A60003FF4D5AF0B0C06BF09044FF0100C4FF02C
:102A7000000C0B0E04BF09020CF1080C0B0F04BF75
:102A800009010CF1040C8B0F04BF89000CF1020C3E
:102A9000CB0F04BF49000CF1010CCCF1200322FA4A
:102AA00003F341EA030102FA0CF2A0EB0C0000F17F
:102AB0000100704723F07F4720F07F4C80EA03003D
:102AC00000F00040ACEB070303F57C5303F1FF0378
:102AD0002DE9804909B44FEA144324EA03484FEA38
:102AE000154B25EA0B4E0FF2042606EB13273E7812
:102AF00003FB0667C7F5000707FB06F64FEAD64655
:102B000006F102064FEA543707FB066CCCF1005C75
:102B10004FEA1C472CEA074C0CFB06F507FB06F4B2
:102B200004EB15464FEA961649085FEA320234BFB5
:102B300000204FF000404FEAD13706FB07FC4FEA78
:102B40001C4C0CFB0BF7D21B03FB0CF761EB0701D2
:102B50000CFB0EF7B0EB074072EB17420CFB08F7CB
:102B600034BFA2EB0742B2EB074261EB17414FEAD9
:102B70000C444FEA910706FB07FC4FEA1C4C0CFB88
:102B80000BF7B0EBC74072EB573203FB0CF734BFC7
:102B9000A2EBC742B2EBC74261EB57310CFB0EF719
:102BA000B0EBC70072EB57720CFB08F734BFA2EB17
:102BB000C702B2EBC70261EB57714FEA816141EA8C
:102BC00092114FEA826242EA90124FEA806004EB6F
:102BD000CC04039F4FEAD13706FB07FC4FEA1C4C9D
:102BE0000CFB0BF7D21B03FB0CF761EB07010CFB93
:102BF0000EF7B0EB074072EB17420CFB08F734BF3F
:102C0000A2EB0742B2EB074261EB17414FEA8C554A
:102C100004EB9C244FEA910706FB07FC4FEA1C4C8F
:102C20000CFB0BF7B0EBC74072EB573203FB0CF712
:102C300034BFA2EBC742B2EBC74261EB57310CFB8A
:102C40000EF7B0EBC70072EB57720CFB08F734BFFE
:102C5000A2EBC702B2EBC70261EB57714FEA816189
:102C600041EA92114FEA826242EA90124FEA806092
:102C700015EB4C2544F100044FEAD13706FB07FC65
:102C80004FEA1C4C0CFB0BF7D21B03FB0CF761EB60
:102C900007010CFB0EF7B0EB074072EB17420CFB81
:102CA00008F734BFA2EB0742B2EB074261EB1741D2
:102CB0004FEA813141EA92414FEA823242EA904240
:102CC0004FEA80304FEA0C7615EB1C1544F10004F6
:102CD00048EA03434EEA0B484FF0000EB2EB080CF3
:102CE00071EB030724BF624639464EEB0E0E4FF0E0
:102CF000000B0018524149414BEB0B0BB2EB080C97
:102D000071EB03077BF1000B24BF624639464EEBA3
:102D10000E0E4FF0000B0018524149414BEB0B0BCC
:102D2000B2EB080C71EB03077BF1000B24BF62468A
:102D300039464EEB0E0E51EA020718BF46F0010667
:102D400016EB0E7655F1000254F1000103D5BDE8F3
:102D50008901BDE80088BDE88901BDE80048B619D1
:102D6000524141EB0101A3F10103704780807F7E56
:102D70007D7C7B7A797877767675747372717170F1
:102D80006F6E6E6D6C6C6B6A6A69686867666665A3
:102D90006464636362616160605F5F5E5E5D5D5C31
:102DA0005C5B5B5A5A5959585857575656555555A2
:102DB0005454535352525251515050504F4F4F4E02
:102DC0004E4D4D4D4C4C4C4B4B4B4A4A4A49494950
:102DD0004848484747474746464645454544444492
:102DE0004443434343424242424141419C46002BBB
:102DF00030D477002BD04FEA37071CB503B44FF01F
:102E000010004FF01001BAF1000F06D0BCF1000F16
:102E1000DCBF40F0080040F008014FF000000FBC9C
:102E2000BDE810400BF1010BBBF1010F08BF5FEAD9
:102E3000170722BF12F1010211F101014FF0004109
:102E400043F1000300F0004043EA00007047F9D36B
:102E50005708D0E746EA06464FEA164613F1400FF8
:102E60001FDD13F1200FDFBF16430A460021203378
:102E70005B42BED0C3F1200746EA06464FEA16463B
:102E800002FA07F746EA070622FA03F2C3F120071F
:102E900001FA07F742EA070221FA03F14FF00003B3
:102EA000A7E746EA020646EA06464FEA164646EA1B
:102EB0000106BCBF46EA0646360C4FF000034FF051
:102EC00000024FF0000194E72DE9804C70B49A465F
:102ED000934691E8380007C831EA400C48BF34EA0D
:102EE000430C03D5FFF7E6FDFFF780FFF0BCBDE81C
:102EF000008C2DE9804C70B49A46934691E83800D6
:102F000007C810F0804F08BF13F0804F03D100F0C6
:102F100005F8FFF76BFFF0BCBDE8008C20F07F47A1
:102F200023F07F4C80EA030000F0004007EB0C0325
:102F3000A3F57C53A3F1FE0392F0000F00F0B380E1
:102F400095F0000F00F077802DE901494FEA11401C
:102F500021EA00484FEA144624EA064700FB06FC33
:102F600008FB06F607FB08F818EB06484CEB164C76
:102F700000FB07F718EB07484CEB17404FEA124BE2
:102F800022EA0B4E4FEA154625EA06470BFB06FCE4
:102F90000EFB06F607FB0EFE1EEB064E4CEB164C28
:102FA0000BFB07F71EEB074E4CEB174B18EB0B0810
:102FB00040F1000018EB0E0B58EB000840F1000048
:102FC0008F1A4FF000014FF000063CBFC943661B4B
:102FD00014BFB5EB040C00213CBFC943F61B4FEAFC
:102FE000174427EA04454FEA1C472CEA074C04FB28
:102FF000076205FB07F70CFB05F616EB074642EBED
:10300000174204FB0CFC16EB0C4642EB1C421BEB7C
:10301000060658EB020241414EEA8E0E46EA9E0633
:1030200001D5BDE80189B619524141EB0101A3F177
:103030000103BDE801894FEA144524EA05464FEA39
:10304000114721EA074C05FB07F406FB07F70CFBC9
:1030500006F111EB074144EB174405FB0CFC11EBA7
:103060000C4144EB1C444FEA124722EA074C05FB93
:1030700007F206FB07F70CFB06F616EB074642EBDA
:10308000174205FB0CFC16EB0C4642EB1C456A187C
:1030900054F1000148BF7047B619524141EB01019C
:1030A000A3F10103704795F0000F37D04FEA1142AA
:1030B00021EA02464FEA144724EA074C02FB07F1D3
:1030C00006FB07F70CFB06F414EB074441EB174132
:1030D00002FB0CFC14EB0C4441EB1C414FEA15477E
:1030E00025EA074C02FB07F506FB07F70CFB06F683
:1030F00016EB074645EB174502FB0CFC16EB0C469E
:1031000045EB1C42121951F1000148BF7047B61936
:10311000524141EB0101A3F1010370474FEA14450D
:1031200024EA05464FEA114721EA074C05FB07F15F
:1031300006FB07F70CFB06F212EB074241EB1741C7
:1031400005FB0CFC12EB0C4251EB1C414FF000064E
:1031500048BF7047921841EB0101A3F1010370478A
:1031600003B401984100009850EAC12018BF042020
:103170004A0D18BF40F0010040F2FF72B2EB515F00
:1031800008BF40F00200012808BF052002B07047C8
:1031900030380A2801D20120704700207047000013
:1031A00010B500290AD00878002807D005487844CF
:1031B000FEF7A6F9002801D0002010BD024878448F
:1031C00010BD0000EA030000E203000010B5002972
:1031D0000AD00878002807D005487844FEF790F90F
:1031E000002801D0002010BD0248784410BD000026
:1031F000DA030000D2030000F1EE100A4FF6FF716F
:10320000C0F2C03120EA010040F04070E1EE100A47
:103210007047FDF763BDFDF797BE0000000000009A
:10322000000000003031323334353637383941420E
:103230004344454640305800303132333435363718
:1032400038396162636465664030780004000008C4
:1032500000000000000000020001000010303132C8
:1032600033343536373839616263646566787000A7
:1032700030313233343536373839414243444546AC
:103280005850000002400000000000A000000000B4
:1032900005400000000000C8000000000C400000D5
:1032A0000000409C00000000194000000020BCBE4F
:1032B0000000000034400000BFC91B8E0000000465
:1032C000B5400000504BCFD06607E2CF01000000B0
:1032D0006C4100003E8251AADFEEA73401000000DD
:1032E000D9420000DCB5A0E23A301F97FFFFFFFF94
:1032F000B4450000FD25A0C8E9A3C14FFFFFFFFFB3
:10330000FF3F00000000008000000000FF3F0000C1
:10331000000000800000000000000000000000002D
:10332000010203040607080952756E74696D652071
:103330006D6F64653A2025733B206564697420676E
:103340005F646364635F636F6E66696720696E20A4
:103350004B65696C2057617463682E0A0052756E64
:1033600074696D6520736572766963652061637445
:103370006976652E206D6F64653D30206D6F6E69D6
:10338000746F722C20312070776D2D746573742CDE
:10339000203220636C6F7365642D6C6F6F702E0A22
:1033A00000555341525433207265746172676574DD
:1033B000207072696E74663A20256C7520626175A2
:1033C000640A00485254494D20444C4C3A2025731D
:1033D0000A0050574D3A20256C7520487A2C2070F1
:1033E0006572696F643D256C7520485254494D20C3
:1033F0007469636B730A0052756E74696D65205051
:10340000574D3A20667265713D256C75487A206487
:103410007574793D256C752F3130303020646561CD
:103420006474696D653D256C7520726973653D2511
:103430006C752066616C6C3D256C75207469636BDE
:10344000730A000A422D47343734452D44504F57F4
:103450003120444344432073746172746572207058
:10346000726F6A6563740A006D6F64653D25732031
:1034700073746174653D2573206661756C743D25B8
:103480007320687274696D3D25732076696E3D25E1
:103490006C756D562069696E3D256C756D412076A1
:1034A0006F75743D256C756D5620647574793D2576
:1034B0006C752F256C752064743D256C752F256CFB
:1034C000750A0053797374656D436F7265436C6F51
:1034D000636B3A20256C7520487A0A006E6F742061
:1034E0007265616479006E6F742D72656164790034
:1034F00073746F707065640076696E20756E6465B4
:1035000072766F6C7461676500766F7574206F7684
:103510006572766F6C74616765006E6F6E650072C0
:10352000756E6E696E6700756E6B6E6F776E006399
:103530006C6F7365642D6C6F6F70006D6F6E697466
:103540006F72006661756C7400696E707574206FBF
:1035500076657263757272656E740070776D2D7426
:1035600065737400687274696D20646C6C20746992
:103570006D656F7574000000C836000800000020FB
:10358000500000003C0200081837000850000020DE
:10359000C80600005C0200081C0000004300000098
:1035A000F8FFFFFF0C0000000E0000000F000000FD
:1035B0002E0000001001000043000000F8FFFFFF94
:1035C0000040404040404040404041414141414036
:1035D00040404040404040404040404040404040EB
:1035E000400502020202020202020202020202027A
:1035F000022020202020202020202002020202027F
:1036000002029090909090901010101010101010D6
:1036100010101010101010101010101002020202E2
:103620000202888888888888080808080808080826
:103630000808080808080808080808080202020222
:10364000400000000000000000000000000000003A
:10365000000000000000000000000000000000006A
:10366000000000000000000000000000000000005A
:10367000000000000000000000000000000000004A
:10368000000000000000000000000000000000003A
:10369000000000000000000000000000000000002A
:1036A000000000000000000000000000000000001A
:1036B000000000000000000000000000000000000A
:1036C00000000000000000000024F40001000000E1
:1036D00000000000400D03006400000084030000AF
:1036E000010000002200000022000000E40C0000A5
:1036F00094110000D80E00002C010000C20100004F
:103700005A000000030000003C000000900100008F
:08371000406A00000000000007
:04000005080001D915
:00000001FF
